:020000040000FA
:100000008316453081007C28B000030EB1000B1D23
:1000100021285F302807031CA80A03184216013064
:100020002F07031CAF0A42191A28990A03199A0AC2
:1000300003199B0AC21821288C0A03198D0A031977
:100040008E0A8B1C23280B1C74280608B300340668
:100050003305B400341E2F28950A0319960AB41EDE
:100060003428970A0319980A341F5A288F0A03194B
:10007000900A0319910A9C0A03199D0A03199E0A02
:100080002208A4002308A5000108A2000C08A30070
:100090005F30280703185928421E5928421142127E
:1000A0009C019D019E019F01A001A10199019A015E
:1000B0009B01A801B41F7228920A0319930A03191D
:1000C000940A421968289F0A0319A00A0319A10A71
:1000D0002908AB002A08AC000108A9000C08AA00F6
:1000E0000130AF003308B400310E8300B00E300E83
:1000F0000B118B100B10090000308500F1308600C9
:100100008312850186010C3084008001840A041F5B
:1001100085288001840A041E8928FF30B4007E22CD
:10012000F8308B008B112208A6002308A7002408B2
:10013000A602031CA7032508A7022908AD002A0868
:10014000AE002B08AD02031CAE032C08AE028B15CB
:100150000D080F39B2008500FB208C1DAD288C19CD
:10016000AF2801302F07031CFA285F302807031C33
:10017000FA2886100030850106158316F5308600B2
:100180008312C21499019A019B0101302F070318B1
:10019000C5280D301B02031CEA2842150C089900E3
:1001A0000D089A000E089B000F089C0010089D0087
:1001B00011089E0012089F001308A0001408A10057
:1001C0008C018D018E018F019001910192019301AB
:1001D0009401F32899019A019B019C019D019E01C4
:1001E0009F01A001A1018316F13086008312061140
:1001F0007E22C2109228861080306822861442190E
:1002000006295C212030682268221029703068227B
:100210007230682265306822763068222030682289
:10022000A221203068226822682293218610C030E3
:10023000682286143B212030682204222030682264
:100240006822EB21861094306822861420306822C0
:10025000682268226822D02120306822CE218610B0
:10026000D43068228614532120306822B3212030F4
:100270006822B12108005F30280703184C2927089D
:10028000BA002608B9005630B7008230B600F52211
:100290009C2242105D2252292030682220306822A0
:1002A0003030682208005F30280703187129693050
:1002B0002F070318812971295F30280703188C291B
:1002C00069302F07031881292E08B7002D08B600C2
:1002D0002708BA002608B900F5229C2242105D22A8
:1002E00092290530B8009D30B7004030B600BB0100
:1002F0002E08BA002D08B90038239C2242105D2236
:1003000092295F30280703188C29663068222D3027
:1003100068226330682292292D3068222D306822AD
:100320002D30682208002E22BD228B111408BB003C
:100330001308BA001208B9008B1538239C22421406
:100340005D2208003722BD228B112108BB00200846
:10035000BA001F08B9008B1538239C2242145D2275
:1003600008004022B4294922BB010E30BA004E30A9
:10037000B90038239C2242105D223A30682240089E
:10038000B8003F08B700B601BB013D30BA000930E4
:10039000B90038239C2242105F2208002E22D12966
:1003A0003722BB010930BA00F430B90038239C224F
:1003B00042105D222E3068224008B8003F08B70086
:1003C000B601BB011930BA007B30B90038239C223A
:1003D00042105F2208002E22BB010330BA005230C7
:1003E000B9003808031DF82940303702031CFE29E4
:1003F0004022382327222E2238231C2ADD224022A5
:100400005222202238231C2A3722BB010330BA0093
:100410005230B9003808031D112A40303702031C3E
:10042000172A492238232722372238231C2ADD2283
:1004300049225222202238239C2242145B220800A7
:100440003E08B8003D08B7003C08B60008003E086A
:10045000BB003D08BA003C08B90008008B11110828
:10046000B8001008B7000F08B6008B1508008B11F4
:100470001E08B8001D08B7001C08B6008B15080040
:100480008B110E08B8000D08B7000C08B6008B15CC
:1004900008008B111B08B8001A08B7001908B6002D
:1004A0008B1508003808BB003708BA003608B900B9
:1004B0000800430868224408682245086822460864
:1004C0006822421C652A2E306822470868220800EC
:1004D000B500350E6F2235086F22350808000F3938
:1004E00010388500000006150000061100003208D3
:1004F00085002830C8000512A22308006430C80017
:100500009523861003306F220530C80095230330F1
:100510006F226430C800A22300306F2202306F22A5
:1005200028306822013068220230C8009523063046
:1005300068220C306822080048308400AA22AA22CF
:10054000AA22AA22AA223030C307C407C507C607B9
:10055000C70708001030C800BE010310BC0DBD0D58
:10056000BE0D0A303E020318BE000318BC0AC80BB9
:10057000AD2A84033E08800008003808BB00370815
:10058000BA003608B9000310B60DB70DB80D031048
:10059000B60DB70DB80D3908B60701300318B70707
:1005A0000318B8073A08B7070318B80A3B08B80792
:1005B0000310B60DB70DB80D08003908BC003A0895
:1005C000BD00BE01BF011030C80003103C1CEE2A64
:1005D0003608BE070318BF0A3708BF07BF0CBE0C9A
:1005E000BD0CBC0CC80BE52A08001030C800390847
:1005F000BF003A08C000BC01BD010310BF0DC00D13
:100600000318082BC80BFE2AC215BF01C001080041
:10061000BF01C0011030C9004808C9020310B60D5F
:10062000B70DBF0DC00DC80B0E2B3A084002031CBE
:10063000292B40083A02031C212B39083F02031CD6
:10064000292B3908BF02031CC0033A08C002031457
:100650002A2B0310BC0DBD0DC9080319362BC90385
:100660000310B60DB70DBF0DC00D152BC21108003C
:100670001830C8003908BF003A08C0003B08C10064
:100680000310BC01BD01BE01BF0DC00DC10D03189B
:10069000502BC80B442BC215BF01C001C10108007B
:1006A000BF01C001C1011830C9004808C9020310C8
:1006B000B60DB70DB80DBF0DC00DC10DC80B572B32
:1006C0003B0841020319672B0318742B832B3A084C
:1006D000400203196E2B0318742B832B39083F0239
:1006E0000319742B031C832B3908BF020130031C30
:1006F000C002031CC1023A08C002031CC1033B082C
:10070000C1020314842B0310BC0DBD0DBE0DC9081E
:100710000319932BC9030310B60DB70DB80DBF0D08
:10072000C00DC10D602BC2110800C90100000000FE
:1007300000000000000000000000C90B962BC80B51
:0A074000952B0800C80BA22B08003F
:02400E00F23F7F
:00000001FF
